:10140000000600205D170000FD1500000516000015
:101410000516000005160000051600000516000060
:101420000516000005160000051600000516000050
:101430000516000005160000051600002D1E000010
:101440000516000005160000051600000516000030
:101450000516000005160000051600000516000020
:101460000516000005160000051600000516000010
:1014700029200000051600000516000005160000D2
:1014800005160000051600000516000005160000F0
:1014900005160000051600000516000005160000E0
:1014A00005160000051600000516000005160000D0
:1014B00005160000051600000516000005160000C0
:10150000FFFFFFFFFFFFFFFFFFFFFFFF87FFFEFF64
:1015100010B5064C2378002B07D1054B002B02D0C9
:10152000044800E000BF0123237010BD08FFFF1F27
:1015300000000000F43C0000084B10B5002B03D065
:101540000749084800E000BF07480368002B00D1A6
:1015500010BD064B002BFBD09847F9E700000000B8
:101560000CFFFF1FF43C000008FFFF1F00000000FD
:1015700020280DDC1F23C217D20E80181840801AB5
:101580001E3BC0218340034A4900535013607047FB
:10159000C046FCE700E100E020280BDC1F23C21757
:1015A000D20E80181840801A1E3B834080220249C8
:1015B0008B507047C046FCE700E100E070B503299E
:1015C00019DC202817DC03242300FF22C5172B4039
:1015D000AD0F1B18084E401904409B10B4468901FA
:1015E000641B134011402240D20091409B00634491
:1015F0001A681143196070BD00E400E010B500F0F6
:10160000F1F810BDFFBE7047104B114A1149D1507F
:10161000114B124A23219A8001225A701970104BE3
:101620009A6106230F4A1370517809330B40002149
:1016300053700D4B1970103113791942FCD00C22E4
:1016400008490B791A42FCD17047C046080D0000CA
:1016500000E000E0001400000020054003E8FFFF68
:1016600000800440004006400050064070210D4AB2
:101670000D4853788B43537013780F318B432339C4
:101680000B431370094A0A4953680B4004210B436A
:101690005360C122074992008B5803408B5062B6B9
:1016A0007047C04600D00740FFFF00FF00800440A5
:1016B000F9FFF7FF00E100E070B503240125002ADF
:1016C0000AD003000B431C4207D1032A05D908C9DD
:1016D000043A08C0002AF4D170BD1D4208D1012A85
:1016E00006D900268B5F023A038002310230E6E71A
:1016F0000B78013A037001310130E0E77047C046D2
:1017000010B5884203D0002A01D0FFF7D5FF10BDE5
:1017100010B50E4C002C16D021686068002909D144
:10172000002811D1A368002B0DD00C34216860680B
:101730000029F5D0A2688142F7D0002AF5D0FFF742
:10174000BBFF0C34F2E710BDA268F6E7143E0000C0
:101750007047C0467047C0467047C04670B5FFF737
:10176000F7FFFFF751FF194B181C002805D08546DD
:1017700081B00020C043009001B0154B154AD21A29
:1017800016D003250124002005E0032A06D902C350
:10179000043A002A0CD029001940F6D02100194043
:1017A0000FD1012A0DD0023A19800233002AF2D15A
:1017B000FFF7AEFFFFF7D0FF0749002002F058F80F
:1017C000FEE71870013A0133E3E7C0460006002047
:1017D00008FFFF1F3802002024FFFF1F10B5FFF78E
:1017E000BDFFC0460221024A53688B4353607047D5
:1017F00000800440002201210220034B1A7059701E
:101800009870D9701A717047F0FFFF1F114B124A80
:1018100012491A60FA2292005A601961104A032094
:1018200020219A600022585415300131585401315A
:101830005A5401315A541438013158542339213043
:1018400019540130DA609A61DA615A611A54273208
:1018500099547047C4FFFF1FF0490200C8010CC42F
:10186000530241000B4B0C499A690A409A6159692D
:101870000A4A0A435A619968094A0A439A605968B0
:10188000084A0A435A60084A084B51680B435360A0
:101890007047C04600F00F40BF0F19FF84000608D4
:1018A00004000600800000080090044000E1E00011
:1018B0007047C0467047C0467047C0460422014B7F
:1018C0009A60704700F00F400422014B5A60704745
:1018D00000F00F400422014BDA60704700F00F4027
:1018E0008022014B9A60704700F00F408022014B2C
:1018F0005A60704700F00F40024B18690006C00F95
:101900007047C04600F00F408022024B12055A601B
:101910007047C04600F00F408022024B12059A60CB
:101920007047C04600F00F40024B18690001C00F1D
:101930007047C04600F00F4001281DD0002813D08A
:10194000022809D0032806D180220F4B92025A6048
:101950008022D2025A60704780220B4B92029A601A
:101960008022D2025A60F6E78022074B92029A60E8
:101970008022D2029A60EEE78022034B92025A60E4
:101980008022D2029A60E6E700F00F4080210B4AE5
:101990008902136812680B408021C9020A40002B9B
:1019A00003D10020002A00D170470220002BFBD079
:1019B0000138002AF8D00230F6E7C04600F00F40A8
:1019C000044B18691B698002C00F5B02DB0F4000EB
:1019D0001843704700F00F40074A136910691269F5
:1019E0009B04DB0F00045204D20F9B00C00F134373
:1019F000400018437047C04600F00F4007282BD81E
:101A0000164B80001B589F46154B18690004C00FE9
:101A10007047134B18698004C00FF9E7104B186921
:101A20004006C00FF4E70E4B1869C004C00FEFE783
:101A30000B4B18690002C00FEAE7094B18698002D6
:101A4000C00FE5E7064B18694002C00FE0E7044B02
:101A500018694004C00FDBE70020D9E7F438000024
:101A600000F00F4001280FD0002808D0022801D034
:101A700000207047074B18684003C00FF9E7054B7B
:101A800018680006C00FF4E7024B1B685B0C184097
:101A9000EFE7C04600F00F4001280CD0002806D028
:101AA000022803D18022064BD2029A60704780221E
:101AB000034B9A60FAE78022014B92029A60F5E7A5
:101AC00000F00F4001280CD0002806D0022803D1D6
:101AD0008022064BD2025A6070478022034B5A6024
:101AE000FAE78022014B92025A60F5E700F00F40BE
:101AF00000207047002070477047C04608211F4AE9
:101B000070B5536880248B4353601D4A0831536974
:101B100000200B43536193691A4910250B409361D0
:101B200000210A23640395601669264201D0013121
:101B3000C9B255601669264201D10130C0B2013BDD
:101B4000DBB2002BEFD10A2912D000220E4B1A7003
:101B500010210B4B5A698A435A61802299695203BA
:101B60000A4308219A61054A53680B43536070BDCC
:101B70000A28EAD10122044B1A70E9E700800440E8
:101B800000F00F40FFFFEFFFC0FFFF1F10B5144B29
:101B900082B01B78002B01D102B010BD01220023BE
:101BA0000221104C6270E2702370A1702371FFF764
:101BB0002DFE00F0CDFA20000B4900F07FFB042041
:101BC00000210A4C0A4AE0600191019B9342FAD835
:101BD000019B01330193019B9342F9D9F3E7C0467E
:101BE000C0FFFF1FF0FFFF1FC4FFFF1F00F00F40EB
:101BF0001FA10700F8B500F013F97B4C2368C01A49
:101C0000632800D8F8BD00F00BF901212060002006
:101C100000F0DAFBC30700D5BBE0744C4023744DE1
:101C2000627829690B409A4209D0012A00D1A7E0C5
:101C30006F21002000F0C8FB002800DA9CE0802122
:101C40006B4A2078136949010B4098420AD0136906
:101C50000B401900481E81412170002B00D088E004
:101C600080339360634B1B79002BCBD08025604978
:101C7000AD030B6901202B405A1E93410A69A678D7
:101C8000920D5B00024013439E421AD00B692B4019
:101C90005A1E93410A695B00920D02401343A370E0
:101CA000022B00D18BE0032B00D193E0012B00D15C
:101CB0008EE00121002000F0EFFC0421002000F064
:101CC000C5FC80274A49BF010B6980253B405E1E49
:101CD000B3419A000B692D022B40581E834101200D
:101CE0000E695B00B60B06401643E27833439A4216
:101CF00027D00A693A40531E9A410B6909692B4063
:101D00005D1EAB41890B0840920002435B00134308
:101D100010210020E37000F057FBE178364BF825E6
:101D20005A5C5B18197A1F2312026D0100030B40E5
:101D30002A40000F00041A4302431021002000F043
:101D400033FB80202A4B22791969000401408A4222
:101D500000D157E71A6902401100481E81412171E4
:101D6000002A25D1802292025A608022D2025A6033
:101D700048E78023536075E72B691B0600D55EE7B3
:101D80001B4B002019694906C90F617000F042FC25
:101D900055E78023164C636000F068FB80239B02AC
:101DA00063608023DB026360FF23104C237035E700
:101DB000802292025A608022D2029A6022E7012198
:101DC000002000F069FC0521002000F03FFC78E7CE
:101DD00000216FE70021002000F05EFC08210020B8
:101DE00000F034FC6DE7C0464CFFFF1F08FEFF1FEC
:101DF00000F00F40F0FFFF1F14390000FA2100220D
:101E0000034BC9011A6059609A6007321A60704723
:101E100010E000E00022014B1A60704710E000E083
:101E2000014B18687047C04650FFFF1F0C4A1368EB
:101E3000013313600B4B1A68002A05D01A68013A67
:101E40001A601B68002B07D0074B1A68002A02D0C3
:101E50001A68013A1A6070470122044B1A70F3E7BE
:101E600050FFFF1FFCFFFF1F00000020F8FFFF1FB7
:101E700010B5FFF7FBFB10BD1D4B70B5040008004B
:101E80009C4225D00C21E3788B43E3700023A370A0
:101E9000072A18D8174B9200D1584B080011C018C8
:101EA00001F05AFC1F212278030A8A430B40134396
:101EB0002C22C0B223706070E3781343E3700C4BA4
:101EC0009C4211D070BD962396215B018901E5E704
:101ED000802309495B03CD682B43CB600023E3706B
:101EE000A370A3716371CDE70C20FFF741FBE9E715
:101EF00000A0064024390000008004400822C37876
:101F00009343C3707047C04610B5020002490348AE
:101F1000FFF7B2FF10BDC0460024F40000A0064049
:101F200010B5054C020005492000FFF7A5FF082267
:101F3000E3789343E37010BD00A006400024F40052
:101F40000B4B10B50400984204D02C22C378934365
:101F5000C37010BD0C20FFF71FFB2C22E37805494E
:101F60009343054AE370D3680B40D360F1E7C04662
:101F700000A00640FFFFEFFF0080044010B50C20DA
:101F8000FFF70AFB2C21054AD3788B43D370044A10
:101F90000449D3680B40D36010BDC04600A0064082
:101FA00000800440FFFFEFFF094A13680133202B34
:101FB0000CD051688B4208D01168511808728021EA
:101FC0001360044AD3780B43D37070470023F0E7C3
:101FD00054FFFF1F00A006400A4B996ADA6A91423B
:101FE0000ED09A6A511C996230219A18525C027084
:101FF0009A6A0120202A00D0704700229A62FBE7EB
:102000000020F9E754FFFF1F034B00201A78002A35
:1020100001D0187001307047F8FFFF1F014B1865A1
:102020007047C04654FFFF1F30B5264B1B79DBB20B
:102030009A0615D5244AD16A0131202936D0906AF2
:10204000814207D030251F4CD06AE4791018E4B2E1
:102050004455D16205201D490860116D1C4A11606C
:1020600040221A4203D01748C1789143C1705BB235
:10207000002B00DB30BD164B19680029FAD1124B3A
:1020800018685A68904216D05A68501C58609A18BE
:10209000127A0C48D2B2C2715A68202A00D1596013
:1020A0004021084AD3780B43D370E3E70021906ABC
:1020B0008142C7D1CEE77F23024AD1780B40D3704B
:1020C000D8E7C04600A0064054FFFF1FFCFFFF1FDB
:1020D0000000002080230D4A1B03D16882B00B430F
:1020E0001C21D3600A4B1A780A431A7011226946E0
:1020F0009A705A79D2B2CA71CA79002240215A70B4
:102100001A780A431A7002B07047C0460080044033
:102110000070074070B50C001500002802D00024A4
:10212000200070BDFFF7F8FB2021084AD378194240
:10213000FCD05471054AD3785BB2002BFBDA54799A
:10214000E4B2002DECD0FFF7DFFBE9E700700740B9
:102150000E4A93795BB2002B00DB704713785B0665
:102160000BD413785BB2002B09DB3F21074A1378AD
:102170008B4330390B431370EFE71378EDE7137897
:102180000F2253409B06E8D1EFE7C0460000024013
:1021900080235B05C05C704730B580248D186405D2
:1021A000002A06D0035D01300B70013180B28D42F0
:1021B000F8D130BD70B5C3070BD48023441CA4B242
:1021C0005B05E55C064B984729002000054B9847C6
:1021D00070BD8023013884B25B05E55C2000F1E727
:1021E00015FEFF1F5DFEFF1F70B50D000400FFF719
:1021F000E1FF29002000014B984770BD5DFEFF1FE5
:10220000F8B54746CE4680B501270F40C903804642
:10221000B9460E0C0DD0040000250B4F20000135EF
:102220000234B847A4B2B542F8D16D004544ABB210
:1022300098464B46002B02D04046FFF7BBFF0CBC34
:1022400090469946F8BDC04615FEFF1FF8B5DE461C
:1022500057464E4645468B46E0B51100170081466D
:10226000FFF7CEFF03233B40BF039A463F0C14D039
:10227000114B5E464C460025984631002000042252
:1022800004340135C047A4B20436BD42F5D1AB00D9
:102290004B449BB29946AD00AB445346002B04D04F
:1022A000524659464846044B98473CBC904699468E
:1022B000A246AB46F8BDC046ADFEFF1F70B51A4B37
:1022C00005001B780C00652B28D07F20FFF772FFDC
:1022D00000217F20154EB047052229000020FFF77E
:1022E000B5FF210028222020FFF7B0FF7F20FFF755
:1022F00061FF65217F20B0470023802252059A1894
:102300001278EA540133052BF7D10023084A9A18B2
:102310001278E2540133282BF8D170BD054B1B789D
:10232000002BE9D0D1E7C0467F0000105DFEFF1F03
:1023300020000010C0FFFF1FF8B5CE46474680B50D
:102340000F008021804691461D0008AB1C78394360
:1023500009AB00221E78FFF7DDFE49464046002209
:10236000FFF7D8FE290040460022FFF7D3FE2100E8
:1023700040460022FFF7CEFE310040460122FFF723
:10238000C9FE4B461B021D437F232D022C433B40BD
:10239000044A240234439B009C500CBC904699464E
:1023A000F8BDC0460400002030B5131483B0150EEC
:1023B000D4B212120194D4B2DBB200942A00FFF717
:1023C000BBFF03B030BDC04670B57F240522254B4E
:1023D0000C401B5D05001A4203D1234BA400E058BA
:1023E00070BD21000022FFF795FE00220021280089
:1023F000FFF790FE002200212800FFF78BFE00224D
:1024000000212800FFF786FE012200212800FFF7A7
:1024100081FE210000222800FFF77CFE002200211F
:102420002800FFF777FE0022060200212800FFF7B0
:1024300071FE0022064300212800FFF76BFE3602E2
:102440000643012200212800FFF764FEDF23360245
:10245000223C30431C42C3D10302C1D5FF231B06DB
:102460001843BDE7443900000400002030B50120C6
:1024700083B0FFF761FAFFF7D3FC0400FFF7D0FC4D
:10248000001BC317C0185840C728F7DD22235F4C34
:102490000020E25C013BE35C12041B021A43202390
:1024A000E35C03251A43130CD1B21212D2B201918C
:1024B000009210210022FFF73FFFA368544A8020BA
:1024C0001A402323A260E15C802349049B02194047
:1024D0002523E35C40051B070340194326231143D2
:1024E0008022E35C92055B07134019432423E25CDE
:1024F0001C3B9B1AF0221B061205134019430A0EBF
:10250000C8B20B140912C9B201900091DBB26C2160
:102510000020FFF711FFE168A37B0A0EC8B2091281
:10252000C9B20190009100206D21FFF705FF2169DC
:10253000A37C0A0EC8B20912C9B201900091002012
:102540007021FFF7F9FE6169A37D0A0EC8B2091276
:10255000C9B20190009100201321FFF7EDFEA1699F
:10256000A37E0A0EC8B20912C9B2019000910020E0
:102570001421FFF7E1FEE169A37F00240A0EC8B22F
:102580000912C9B20190009100201521FFF7D4FE75
:10259000019400940023002220210020FFF7CCFEAC
:1025A00001940094002300222D210020FFF7C4FE97
:1025B000019400940023002221210020FFF7BCFE9B
:1025C0000723009401930022002301210020FFF73C
:1025D000B3FE019500940023002200210020FFF7A4
:1025E000ABFE062300950193002200230921002061
:1025F000FFF7A2FE0A23009401930022093B0A215F
:102600000020FFF799FE03B030BDC046C4FFFF1F96
:10261000FFFFFDE030B50D0083B000210400FFF79F
:10262000D3FE0421084BAD00294018400843030C99
:10263000C2B20012C0B2019200900022002120001C
:10264000FFF77AFE03B030BDFBFF030030B50C008E
:1026500083B06C210500FFF7B7FEF02324061B05AD
:102660001C40084B18402043020EC1B20314001254
:10267000C0B201910090DBB26C212800FFF75CFE34
:1026800003B030BDFFFFFFF010B56C21FFF79CFEDB
:102690000001000F10BDC04630B50C0083B06C21A6
:1026A0000500FFF791FE802324075B051C40084BC3
:1026B00018402043020EC1B203140012C0B20191AF
:1026C0000090DBB26C212800FFF736FE03B030BD6E
:1026D000FFFFFFEF10B56C21FFF776FEC000C00FC3
:1026E00010BDC04630B50C0083B06C210500FFF76B
:1026F0006BFE802364079B051C40084B1840204359
:10270000020EC1B203140012C0B201910090DBB2FC
:102710006C212800FFF710FE03B030BDFFFFFFDF84
:1027200010B56C21FFF750FE8000C00F10BDC046F1
:1027300030B50D0083B06C210400FFF745FE002D7D
:102740000FD10A4B1840020EC1B203140012C0B2DE
:1027500001910090DBB26C212000FFF7EDFD03B08A
:1027600030BD80239B021843EDE7C046FFFFFDFF0D
:1027700010B56C21FFF728FE8003C00F10BDC046C6
:1027800030B50C0083B06D210500FFF71DFE6023FE
:1027900064011C4098432043020EC1B2031400128E
:1027A000C0B201910090DBB26D212800FFF7C4FD9B
:1027B00003B030BD30B50C0083B06D210500FFF7CC
:1027C00003FEC0236403DB011C40084B1840204378
:1027D000020EC1B203140012C0B201910090DBB22C
:1027E0006D212800FFF7A8FD03B030BDFF9FFFFF5C
:1027F00030B50C0083B06D210500FFF7E5FDF02337
:1028000024021B011C40084B18402043020EC1B299
:1028100003140012C0B201910090DBB26D212800B8
:10282000FFF78AFD03B030BDFFF0FFFF30B50D00AC
:1028300083B06D210400FFF7C7FD0F2188432940B5
:102840000843020EC1B203140012C0B201910090FD
:10285000DBB26D212000FFF76FFD03B030BDC04635
:1028600030B50C0083B06D210500FFF7ADFD084BBE
:10287000184023041843020EC1B20012C0B20191E5
:1028800000901B0C6D212800FFF756FD03B030BDF2
:10289000FFFF00FF30B50D0083B06D210400FFF78E
:1028A00093FD002D0FD10A4B1840020EC1B2031444
:1028B0000012C0B201910090DBB26D212000FFF741
:1028C0003BFD03B030BD80231B021843EDE7C0463B
:1028D000FF7FFFFF30B50D0083B06D210400FFF7CF
:1028E00073FD002D0FD10A4B1840020EC1B2031424
:1028F0000012C0B201910090DBB26D212000FFF701
:102900001BFD03B030BD80235B041843EDE7C046D8
:10291000FFFFFFFE10B56D21FFF756FD4006800F4B
:1029200010BDC04610B56D21FFF74EFD4004800F6D
:1029300010BDC04610B56D21FFF746FD0005000F24
:1029400010BDC04610B56D21FFF73EFD0F231840A6
:1029500010BDC04610B56D21FFF736FD0314FF20F2
:1029600018401B0601D5014B184310BD00FFFFFFA7
:1029700010B56D21FFF728FD0004C00F10BDC04643
:1029800010B56D21FFF720FDC001C00F10BDC0467E
:1029900070B57A4C63784B2B00D1A1E010D9842B11
:1029A00000D1A9E000D87DE0F02B68D0FF2B00D04B
:1029B000ACE00A2800D1BAE0092800D1AEE070BD31
:1029C000412B00D180E061D9422B49D0432B00D06C
:1029D0009CE00A2800D1C5E00928F0D1684D217992
:1029E0002B79002B37D0002935D12223654E1031A9
:1029F000F25C013BF35C12041B021A432023F35CDC
:102A000000201A43FFF7D0FC2323F25C80235204FA
:102A10009B021A4025238021F35C49051B070B40CC
:102A20001A43B36880211A432623F35C89055B07A8
:102A30000B401A432423F15C1C3B5B1AF0211B065C
:102A400009050B401A436C210020FFF7ADFC032061
:102A5000FEF772FF217904202971FFF7C5FBAEE76D
:102A60000A285FD00928AAD1454B61689A7891421B
:102A700050D0217908385970FFF7B6FB9FE70A2834
:102A80009DD1414B1A78414B5A6098E7402B3DD17C
:102A90000A286CD0092800D091E721797630FFF719
:102AA000A3FB8CE74C2B31D10A2856D0092800D043
:102AB00085E7334B61685A7891422BD021790738EA
:102AC0009970FFF791FB7AE70A283CD0092800D0DB
:102AD00075E721792A4B00201970FFF785FB6EE717
:102AE0000A282BD0092800D069E72179244B063821
:102AF000D970FFF779FB62E70A2829D0092800D0AE
:102B00005DE7224B5A68224B1A6058E703221F4B9D
:102B10001A7054E704221D4B1A7050E722791D4B9E
:102B20001A704CE7164B5A78184B5A6047E7194B06
:102B30001B785A1E9341154A536040E7104BDA78D0
:102B4000124B5A603BE70E4B1A78104B5A6036E72F
:102B50000F4B1A680D4B5A6031E7094B9A780B4BB3
:102B60005A602CE7064B1A79084B5A6027E77530F4
:102B7000FFF70EFB054B586021E7C046040200201A
:102B8000F0FFFF1FC4FFFF1FECFFFF1F2802002004
:102B90001C020020190200200023034A1370034A7C
:102BA0001370034A137070470C02002020020020AB
:102BB0001902002030B5BC4C83B0A378002B09D19A
:102BC0006378063BDBB2C82B00D99BE1B74A9B0078
:102BD000D3589F460422B64B1A7003B030BD052867
:102BE00000D18FE10628F8D16F210020FFF7ECFB20
:102BF000AF4A83059B0D5360EFE7052800D1D4E170
:102C0000062800D14BE2072800D18FE20828E4D142
:102C10002123A84AD25CA64B5A60DEE7052800D1E2
:102C200006E2062800D15AE2072800D16EE2082801
:102C3000D3D120239F4AD25C9D4B5A60CDE7052813
:102C400000D1E4E1062800D140E2072800D17DE26E
:102C50000828C2D12223974AD25C954B5A60BCE720
:102C60000628BAD112210020FFF7AEFB904B586026
:102C7000B3E7052800D16AE1062800D162E1072800
:102C800000D1AFE20828A8D18B4D042229002C30B6
:102C9000FFF782FA2A68A0781321FFF785FB2A68DC
:102CA000834B5A6099E7052800D12FE1062800D10F
:102CB000B6E2072800D1C1E2082800D08DE77D4B9D
:102CC000DA697B4B5A6088E7052800D183E1062842
:102CD00000D12DE1072800D18EE2082800D07CE742
:102CE000764D042229002830FFF756FA2A68A0788A
:102CF0007021FFF759FB2A686D4B5A606DE7052874
:102D000000D171E1062800D117E1072800D17DE24A
:102D1000082800D061E76A4D042229002030FFF71F
:102D20003BFA6C21A078FFF74FFB2A68654B6C21BA
:102D30001340654A2B6002401A43A078FFF734FB2A
:102D40002A685B4B5A6048E7052800D116E106283F
:102D500000D1ADE1072800D124E2082800D03CE7EB
:102D60002423544AD25C524B5A6036E7052800D1DE
:102D700011E1062800D030E70020FFF7DBFD4C4BC7
:102D800058602AE7052800D10AE1062800D024E788
:102D90000020FFF7D7FD464B58601EE7052800D1FD
:102DA00050E1062800D018E70020FFF7E9FD404B6E
:102DB000586012E7052800D154E1062800D162E1ED
:102DC000072800D1D2E1082800D006E72523394A98
:102DD000D25C374B5A6000E7052800D1D6E00628C0
:102DE00000D0FAE60020FFF7B5FD314B5860F4E65D
:102DF000052800D186E0062800D0EEE66F210020ED
:102E0000FFF7E2FA2A4AC302DB0E5360E5E6052823
:102E100000D184E0062800D109E2072800D12BE286
:102E2000082800D0D9E6234B9A69214B5A60D4E692
:102E3000052800D110E1062800D11DE1072800D1A6
:102E4000C0E1082800D0C8E61A4BDA68184B5A606F
:102E5000C3E6052800D187E0062800D0BDE60020A3
:102E6000FFF758FD124B5860B7E6052800D1FEE089
:102E7000062800D0B1E60020FFF77AFD0C4B586021
:102E8000ABE6052800D1E2E0062800D101E10728E1
:102E900000D179E1082800D09FE62323054AD25CBF
:102EA000034B5A6099E6C04604020020C439000072
:102EB00028020020C4FFFF1FD8FFFF1FD4FFFF1F01
:102EC000CCFFFF1FFFFFFDE00000021F052850D0D0
:102ED000062800D1F4E0072800D109E1082800D035
:102EE0007BE62623DD4AD25CDD4B5A6075E6052879
:102EF0006CD0062800D070E60020FFF713FDD84BF9
:102F000058606AE60322D64B1A7066E66268002AA9
:102F100000DA5FE615210020FFF746FA5DE66268F9
:102F2000002A00DA56E614210020FFF73DFA54E6A5
:102F3000CA4B1A69CA4B5A604FE6C84B9A68C84BCD
:102F40005A604AE6C54B5A69C54B5A6045E6636804
:102F500013211A03120B0020FFF726FA6368BF4AF9
:102F60001B031B0B536138E621790020FFF708FC97
:102F700033E621790020FFF7B5FB2EE608216368D0
:102F80000020C91AC9B2FFF761FB26E621790020AB
:102F9000FFF766FC21E621790020FFF729FC1CE6FB
:102FA00021790020FFF742FC17E610210020FFF7EF
:102FB0000BFA0200D2B2030CA07801922279DBB2A4
:102FC000009210210022FFF7B7F906E621790020D0
:102FD000FFF7F0FB01E6626870210020FFF7E4F9DB
:102FE00062689E4B1A61F8E56C210020FFF7ECF94E
:102FF00062689C4B6C2113409B4A636002401A43F9
:10300000A078FFF7D1F96268944B9A60E5E510214A
:103010000020FFF7D9F902002379A078D1B2120A73
:10302000D2B20191009210210022FFF785F9D4E578
:1030300010210020FFF7C8F9030C0200DBB2A078D2
:103040002179ECE721790020FFF744FCC5E52179DF
:103050000020FFF76DFBC0E562686D210020FFF7DF
:10306000A3F9BAE521790020FFF716FBB5E5217930
:103070000020FFF70FFCB0E56D210020FFF7A4F959
:10308000774B5860A9E50020FFF724FB744B58608C
:10309000A3E50020FFF76CFB714B58609DE5102104
:1030A0000020FFF791F96E4A03041B0E536094E56C
:1030B0000020FFF7E9FA0823181A694B58608CE5DD
:1030C0000020FFF72DFB664B586086E5102100209D
:1030D000FFF77AF9624A03021B0E53607DE5102167
:1030E0000020FFF771F9FF2318405D4B586074E52D
:1030F0000020FFF715FB2624584D010028554620D7
:10310000FFF772F82A5D564B5A6066E510210020E1
:10311000FFF75AF91F212024504D01404020295526
:10312000FFF762F82A5D4E4B5A6056E510210020E9
:10313000FFF74AF92124494DC104C90E4120295500
:10314000FFF752F82A5D464B5A6046E510210020F1
:10315000FFF73AF92224414D0103090F4220295576
:10316000FFF742F82A5D3E4B5A6036E50020FFF734
:10317000B1FA2524394D010028554520FFF734F8D0
:103180002A5D374B5A6028E50020FFF7F1FA232427
:10319000324D010028554320FFF726F82A5D304BB9
:1031A0005A601AE50020FFF76FFA082124242B4DFE
:1031B000091AC9B244202955FFF716F82A5D284B91
:1031C0005A600AE56D210020FFF7FEF8234C042227
:1031D0002100E0600C312C20FFF738F8E268204B2A
:1031E0005A60FAE4214C042221002D30FFF72EF81A
:1031F00022681B4B5A60F0E41D4C04222100293048
:10320000FFF724F82268164B5A60E6E4194C0422B2
:1032100021002130FFF71AF82268114B5A60DCE4D4
:1032200015210020FFF7D0F80D4B5860D5E414218C
:103230000020FFF7C9F80A4B5860CEE415210020A2
:10324000FFF7C2F8054C04222100E0611C313C204C
:10325000FEF7FCFFE269024B5A60BEE4C4FFFF1FA9
:1032600028020020FFFFFDE00000021FD8FFFF1F23
:10327000D4FFFF1FCCFFFF1F14210020FFF7A4F88D
:10328000054C04222100A06118313820FEF7DEFF32
:10329000A269024B5A60A0E4C4FFFF1F280200206D
:1032A00010B5054B9B78002B02D1FFF771FB10BDC9
:1032B0000422024B1A70FAE70402002028020020C0
:1032C00010B5094B9A78022A06D15A685878002A14
:1032D00006D1FEF7E1FB02E00422044B1A7010BD98
:1032E000FEF7F0FBFBE7C0460402002028020020A6
:1032F00010B50B4B9A78002A0BD0022A03D0042277
:10330000084B1A7010BD5878FEF7ACFB054B58609F
:10331000F8E75878FEF772FB024B5860F2E7C046B8
:103320000402002028020020194B5B78002B10D1EA
:103330000122184B18481A70184B9B780370184BD1
:103340001A68002311780133C1540132082BF9D1D6
:103350007047012B12D0022BFAD101220D4B0E48DF
:103360001A700E4B0F499B78037000235A1C083BC0
:10337000CB5C83541300082AF8D1E9E704210A4AF8
:10338000D17153713031013391711371E0E7C0464F
:10339000040200200D02002010020020F0FFFF1F99
:1033A00010FEFF1F00140000280200200249034BFA
:1033B000034AD1507047C0460400FA050C0D0000C6
:1033C00000E000E0124A134B116810B50B4012499F
:1033D0008B4203D00422114B1A7010BD104B52685F
:1033E0009A42F7D1FEF782FA72B6FEF713FD012278
:1033F00080210C4B52425A500131FF315A500A4A37
:103400000A4B0B491A600B4B0B4AD150E5E7C046FB
:103410000402002000FFFF0000819200280200202B
:10342000D6C5B4A300E100E07856341200FEFF1FB9
:103430000400FA050C0D000000E000E0642110B566
:10344000264B274A197010785168587059600E2819
:103450003DD009D9892824D012D80F281ED0882819
:1034600032D1FFF761FF0AE005282DD3082812D9D1
:103470000A2829D89278002A2CD004221A7010BD6C
:10348000F2281ED0FF281FD1164B9942F7D10122F6
:10349000154B1A70F3E7FFF78DFBF0E7FFF728FFF6
:1034A000EDE7FEF7A7F9FEF7B1F901220F4B10493E
:1034B00010481A70FEF702FF0F49104B104AD15006
:1034C000DDE7FFF77FFFDAE702221A70D7E7FFF7A1
:1034D000F7FED4E7FFF75CFAD1E7C04628020020E8
:1034E00004020020D20400000C020020C0FFFF1FD5
:1034F000C4FFFF1FF0FFFF1F0400FA050C0D0000C2
:1035000000E000E0F0B5C64600B5704B82B01B7815
:10351000002B0CD0FB226E4B1B78991F114206D05A
:10352000EB3A93430F2B02D06A4C6B4D06E0694C8B
:103530002378032B46D0042B59D0674D00232370EA
:103540002B70664B1B78002B03D06549654B664A90
:10355000D1506B46D81DFEF73FFD00280ED12378D1
:1035600004221900914305D0FD22063B134201D0ED
:10357000FFF764FF02B004BC9046F0BDFEF744FDC7
:1035800000282ED169466278C979531CDBB2A21893
:1035900063701171092BE2D1544B607021795B7813
:1035A0008B42DCD100230022201D00E0115CCB18EF
:1035B0000132DBB2082AF9D1227B9A426DD0042372
:1035C0002370D7E7444D2B78002B37D0012BB5D192
:1035D0000026474FB85D0136FEF7E6FC092EF9D10B
:1035E000ACE7012363706B46DB792371B7E70023F7
:1035F0000122404D3D4F6B702A706B60B8787E7829
:103600008619FEF7D1FC7878FEF7CEFC2878FEF715
:10361000CBFC6878FEF7C8FCE879FEF7C5FCA87912
:10362000FEF7C2FC01366879FEF7BEFCF6B22879D7
:10363000FEF7BAFC3000FEF7B7FC7EE72B4B2D4FB0
:10364000984698785E783B788619F6187B78F61855
:10365000FB79F618BB79F6187B79F6183B79F618E2
:10366000FEF7A2FC43465878FEF79EFC3878FEF73A
:103670009BFC7878FEF798FCF879FEF795FCB87912
:10368000FEF792FC7879FEF78FFCF6B23879FEF7F8
:103690008BFC3000FEF788FC50E70D4B62791A7006
:1036A000A2795A70E2799A70227ADA71627A9A7102
:1036B000A27A5A71E27A1A71FEF7B2FB00220E4B1F
:1036C00018600E4B1A700323237051E71902002073
:1036D00004020020A8FFFF1F0D0200200C020020A2
:1036E0000400FA050C0D000000E000E0F0FFFF1FF1
:1036F00010020020280200202402002030020020B6
:10370000044A054B52689A4202D10122034B1A70B7
:103710007047C04604020020D20400000C020020C2
:1037200070B5FEF77DFBFA220A4C050023685200B3
:10373000C31A934207D96368002B05D1FEF7C4F87A
:1037400001232560636070BDFEF7B8F80023256093
:103750006360F8E7B8FFFF1F002243088B4274D371
:1037600003098B425FD3030A8B4244D3030B8B4282
:1037700028D3030C8B420DD3FF22090212BA030C8B
:103780008B4202D31212090265D0030B8B4219D36C
:1037900000E0090AC30B8B4201D3CB03C01A52418C
:1037A000830B8B4201D38B03C01A5241430B8B42D4
:1037B00001D34B03C01A5241030B8B4201D30B03BD
:1037C000C01A5241C30A8B4201D3CB02C01A5241E4
:1037D000830A8B4201D38B02C01A5241430A8B42A7
:1037E00001D34B02C01A5241030A8B4201D30B0290
:1037F000C01A5241CDD2C3098B4201D3CB01C01AAA
:10380000524183098B4201D38B01C01A52414309B3
:103810008B4201D34B01C01A524103098B4201D3A1
:103820000B01C01A5241C3088B4201D3CB00C01A0E
:10383000524183088B4201D38B00C01A5241430886
:103840008B4201D34B00C01A5241411A00D20146AB
:10385000524110467047FFE701B5002000F006F81E
:1038600002BDC0460029F7D076E770477047C046D2
:1038700010B5FEF7FDFAFEF7C1FAFDF7BBFFFDF745
:10388000C5FFFDF7EFFF174C2378002B21D0FEF783
:103890007DF9FEF71FFC0122134B1A70FEF758FC4E
:1038A000124C13492000FEF709FD2078FEF72CFB8F
:1038B000FFF772F9FEF71AF8FEF7D8FD0320FEF7BE
:1038C0003BF8FFF72DFF0120FFF71CFEFEF792F9F2
:1038D000F7E7FEF713F92378002BD8D1FEF70EF99E
:1038E000D5E7C046C0FFFF1FECFFFF1FF0FFFF1F23
:1038F000C4FFFF1F1C1A0000261A0000301A000027
:103900003A1A0000441A00004E1A0000081A00007B
:10391000121A0000181A14111B140E0803040303D2
:10392000040403028025000040380000004B000022
:10393000807000000096000000E10000002C0100F3
:1039400000C20100030101020702000000000000A4
:10395000000000000202010202020000000000005C
:10396000000000000303010202020202020202023E
:103970000203000000000002030100000303020133
:103980000100000000000000000000000000000036
:103990000000000000000000000000000000000027
:1039A0000000000002020202020202020202010101
:1039B00003020201020102010000000000000000F9
:1039C00000000000FA2B00001C2C0000042F000057
:1039D0003E2C0000042F0000042F0000042F0000E4
:1039E000042F0000042F0000042F0000042F00000B
:1039F000042F0000042F0000042F0000042F0000FB
:103A0000042F0000A62C0000042F0000042F00004B
:103A1000042F0000042F0000042F0000042F0000DA
:103A2000042F0000042F0000042F0000042F0000CA
:103A3000042F0000042F0000042F0000042F0000BA
:103A4000042F0000042F0000042F0000042F0000AA
:103A5000042F0000042F0000042F0000042F00009A
:103A6000042F0000042F0000042F0000042F00008A
:103A7000042F0000042F0000042F0000042F00007A
:103A8000042F0000042F0000042F0000042F00006A
:103A9000042F0000042F0000042F0000042F00005A
:103AA000042F0000042F0000042F0000042F00004A
:103AB000042F0000042F0000042F0000042F00003A
:103AC000042F0000042F0000042F0000042F00002A
:103AD000042F0000042F0000042F0000042F00001A
:103AE000042F0000042F0000042F0000042F00000A
:103AF000042F0000042F0000042F0000042F0000FA
:103B0000042F0000042F0000042F0000042F0000E9
:103B1000042F0000042F0000042F0000042F0000D9
:103B2000042F0000042F0000042F0000042F0000C9
:103B3000042F0000042F0000042F0000042F0000B9
:103B4000042F0000042F0000042F0000042F0000A9
:103B5000042F0000042F0000042F0000042F000099
:103B6000042F0000042F0000042F0000042F000089
:103B7000042F0000042F0000042F0000042F000079
:103B8000042F0000042F0000042F0000042F000069
:103B9000042F0000042F0000042F0000042F000059
:103BA000042F0000042F0000042F0000042F000049
:103BB000042F0000042F0000042F0000042F000039
:103BC000042F0000042F0000602C0000722C000065
:103BD000C82C0000302E0000FE2C0000482D0000F4
:103BE000B42D0000CC2E0000042F0000042F000094
:103BF000042F0000042F0000042F0000042F0000F9
:103C0000042F0000042F0000042F0000042F0000E8
:103C1000042F0000042F0000042F0000042F0000D8
:103C2000042F0000042F0000042F0000042F0000C8
:103C3000042F0000042F0000042F0000042F0000B8
:103C4000042F0000042F0000042F00006A2E000043
:103C5000EE2E00006C2D0000522E0000842D00007E
:103C60009C2D0000D82D0000042F0000042F000020
:103C7000042F0000042F0000822E0000F02D000011
:103C8000042F00000E2E0000042F0000042F00005F
:103C9000042F0000042F0000042F0000042F000058
:103CA000042F0000042F0000042F0000042F000048
:103CB000042F0000042F0000042F0000042F000038
:103CC000042F0000042F0000042F0000042F000028
:103CD000042F0000042F0000042F0000042F000018
:103CE000042F0000DE2B00003130373656313032E1
:103CF00000000000F8B5C046F8BC08BC9E467047FE
:0C3D0000F8B5C046F8BC08BC9E467047F1
:043D0C003915000065
:043D10001115000089
:103D1400FFFFFFFFFF000000E83C000080235B057D
:103D24009C46604472B630230D4A937193795BB21A
:103D3400002BFBDA0023122193709172D3720133AA
:103D44009370030ADBB293728023C0B2D072937172
:103D5400034A93795BB2002BFBDA62B67047C04624
:103D64000000024080235B059C4610B5604472B697
:103D740030230F4A937193795BB2002BFBDA002353
:103D8400112493709472D37201339370030ADBB2DB
:103D940093720223C0B2D07293707E33D172937146
:103DA400034A93795BB2002BFBDA62B610BDC046BE
:103DB40000000240531E30B5032B25D880235B0539
:103DC4009C46604472B63023104C1125A371002325
:103DD400A370A572E3720133A370030ADBB2C0B20D
:103DE400A372E07202230020A3700D5C0133013042
:103DF400E572DBB29042F7DB8023044AA371937926
:103E04005BB2002BFBDA62B630BDC0460000024054
:103E1400143D000008FEFF1F000100000000000028
:083E2400000000000000000096
:020000041FFFDC
:04FE000000000000FE
:040000030000175D85
:00000001FF
